:1000000045C0000060C000005EC000005CC0000091
:100010005AC0000058C0000056C0000054C0000084
:1000200052C0000050C00000DDC000004CC0000005
:100030004AC0000048C0000046C0000044C00000A4
:1000400042C0000040C000003EC000003CC00000B4
:100050003AC0000038C0000036C0000034C00000C4
:1000600032C0000030C000002EC000002CC00000D4
:100070002AC0000028C0000026C0000024C00000E4
:1000800022C0000020C000001EC0000011241FBEBE
:10009000CFEFD0E1DEBFCDBF11E0A0E0B1E0E2E202
:1000A000F9E000E00BBF02C007900D92AA30B10743
:1000B000D9F721E0AAE0B1E001C01D92AC30B2074F
:1000C000E1F729D12CC49CCF9BB321E030E002C0E2
:1000D000220F331F8A95E2F7292B2BBB08959BB380
:1000E00021E030E002C0220F331F8A95E2F720950D
:1000F00029232BBB089586E090E0E6DF83EC99E0AE
:100100000197F1F700C0000086E090E0E8DF83ECA3
:1001100099E00197F1F700C000000895CF93C82F30
:1001200085BB84E090E0D0DFE6DFC295C07FC5BB31
:1001300084E090E0C9DFDFDFCF910895CF93C82F2F
:1001400085BB84E090E0CBDFD6DFC295C07FC5BB26
:1001500084E090E0C4DFCFDFCF91089581E0EEDF4F
:1001600087E893E10197F1F700C0000080E8E6CF4F
:100170000895CF938FEF84BB85BB8ABB15BA1BBA9A
:10018000C0E2C5BBB8DFC5BBB6DF80E885BBB3DF67
:1001900015BAB1DF80EF85BBAEDF15BAACDF80E604
:1001A00085BBA9DF82E0CADFA6DFCF910895CF9398
:1001B000DF93EC0102C0B2DF219688818111FBCF71
:1001C000DF91CF91089520E030E008C0EFECF7E038
:1001D0003197F1F700C000002F5F3F4F2817390714
:1001E000ACF308951F920F920FB60F9211240BB625
:1001F0000F92CF92DF92EF92FF920F931F932F9364
:100200003F934F935F936F937F938F939F93AF939E
:10021000BF93EF93FF93CF93DF93CDB7DEB7CDB608
:10022000DEB68091000184BD80910A0190910B019E
:10023000019690930B0180930A0190DF80910A014F
:1002400090910B0101969F938F930F2EF2E0EF2E6A
:10025000F1E0FF2EF02DFF92EF921F921F921F925E
:100260001F9274D001962DB73EB7285F3F4F0FB64F
:10027000F8943EBF0FBE2DBF281B390B0FB6F89464
:100280003EBF0FBE2DBF0DB71EB70F5F1F4F209192
:100290000A0130910B012F5F3F4F3F932F93FF9245
:1002A000EF929F938F931F930F9350D0802F912F96
:1002B0007EDF8DB79EB708960FB6F8949EBF0FBE2F
:1002C0008DBF0FB6F894DEBE0FBECDBEDF91CF91CD
:1002D000FF91EF91BF91AF919F918F917F916F911E
:1002E0005F914F913F912F911F910F91FF90EF9050
:1002F000DF90CF900F900BBE0F900FBE0F901F900E
:1003000018958091000184BD87B7806487BF789479
:1003100087E085BD089581B38F7781BB8FEF8ABB5E
:1003200087BB27DF8FE19EE40197F1F700C0000053
:1003300015DF85E091E03BDFE4DF84B58BBB809186
:100340000A0188BB8AE090E03EDFF7CF0F931F934E
:10035000CF93DF93CDB7DEB72E970FB6F894DEBFFD
:100360000FBECDBF0D891E898F89988D26E02C8305
:100370001A83098397FF02C080E090E801979E836B
:100380008D83AE01455E5F4F698D7A8DCE010196FA
:1003900019D04D815E8157FD0AC02F8138854217E3
:1003A00053070CF49A01F801E20FF31F10822E9606
:1003B0000FB6F894DEBF0FBECDBFDF91CF911F9176
:1003C0000F9108952F923F924F925F926F927F927A
:1003D0008F929F92AF92BF92CF92DF92EF92FF9255
:1003E0000F931F93CF93DF93CDB7DEB72B970FB645
:1003F000F894DEBF0FBECDBF6C017B018A01FC010A
:1004000017821682838181FFBFC1CE0101963C0114
:10041000F6019381F70193FD859193FF81917F010F
:10042000882309F4ADC1853239F493FD859193FF9A
:1004300081917F01853221F4B60190E0D6D1E8CFD9
:10044000912C212C312CFFE1F315D8F08B3279F06F
:1004500038F4803279F08332A1F4232D20611DC05D
:100460008D3261F0803369F4232D216016C0832D15
:100470008260382EE32DE4603E2E2AC0F32DF86012
:100480001DC037FC2DC020ED280F2A3040F08E32E1
:10049000B9F436FC75C1232D2064322E19C036FE06
:1004A00006C08AE0989E200D1124922E11C0EAE029
:1004B0002E9E200D1124222EF32DF0623F2E08C017
:1004C0008C3621F4832D8068382E02C0883641F4A2
:1004D000F70193FD859193FF81917F018111B3CF46
:1004E000982F9F7D9554933028F40C5F1F4F9FE306
:1004F00099830DC0833631F0833771F0833509F06D
:1005000055C020C0F801808189830E5F1F4F882469
:100510008394912C530112C02801F2E04F0E511C1C
:10052000F801A080B18036FE03C0692D70E002C0E2
:100530006FEF7FEFC5014ED14C018201F32DFF77A4
:100540003F2E15C0280122E0420E511CF801A08068
:10055000B18036FE03C0692D70E002C06FEF7FEFFF
:10056000C5012DD14C01F32DF0683F2E820133FCE3
:1005700019C0822D90E088169906A0F4B60180E299
:1005800090E033D12A94F5CFF50137FC859137FE01
:1005900081915F01B60190E028D121102A9421E0D9
:1005A000821A91088114910479F7E1C0843611F020
:1005B000893639F5F80137FE07C060817181828183
:1005C00093810C5F1F4F08C060817181072E000C62
:1005D000880B990B0E5F1F4FF32DFF763F2E97FF71
:1005E00009C090958095709561957F4F8F4F9F4F73
:1005F000F0683F2E2AE030E0A30133D1882E861820
:1006000044C0853731F4232D2F7EB22E2AE030E00E
:1006100025C0932D997FB92E8F36C1F018F48835F7
:1006200079F0AEC0803719F0883721F0A9C0E92FE2
:10063000E061BE2EB4FE0DC0FB2DF460BF2E09C0DC
:1006400034FE0AC0292F2660B22E06C028E030E012
:1006500005C020E130E002C020E132E0F801B7FE41
:1006600007C060817181828193810C5F1F4F06C03A
:100670006081718180E090E00E5F1F4FA301F1D097
:10068000882E8618FB2DFF773F2E36FE0DC0232DBA
:100690002E7FA22E891458F434FE0BC032FC09C000
:1006A000832D8E7EA82E05C0B82CA32C03C0B82C99
:1006B00001C0B92CA4FE0FC0FE01E80DF11D808120
:1006C000803321F49A2D997EA92E09C0A2FE06C07E
:1006D000B394B39404C08A2D867809F0B394A3FC34
:1006E00010C0A0FE06C0B21480F4280C922C9B18F7
:1006F0000DC0B21458F4B60180E290E076D0B39405
:10070000F8CFB21418F42B1802C0982C212CA4FE98
:100710000FC0B60180E390E068D0A2FE16C0A1FC35
:1007200003C088E790E002C088E590E0B6010CC005
:100730008A2D867851F0A1FE02C08BE201C080E2D2
:10074000A7FC8DE2B60190E050D0891430F4B601D8
:1007500080E390E04AD09A94F8CF8A94F301E80DB0
:10076000F11D8081B60190E040D08110F6CF2220AB
:1007700009F44ECEB60180E290E037D02A94F7CF4C
:10078000F6018681978102C08FEF9FEF2B960FB6FF
:10079000F894DEBF0FBECDBFDF91CF911F910F91B7
:1007A000FF90EF90DF90CF90BF90AF909F908F9091
:1007B0007F906F905F904F903F902F900895FC0135
:1007C0000590615070400110D8F7809590958E0F7C
:1007D0009F1F0895FC016150704001900110D8F7EF
:1007E000809590958E0F9F1F08950F931F93CF9321
:1007F000DF93FB01238121FD03C08FEF9FEF2CC00E
:1008000022FF16C046815781248135814217530744
:1008100044F4A081B1819D012F5F3F4F318320833C
:100820008C93268137812F5F3F4F3783268314C0F7
:100830008B01EC01FB010084F185E02D0995892BEA
:10084000E1F6D80116968D919C911797019617960F
:100850009C938E931697CE01DF91CF911F910F91AC
:100860000895FA01AA27283051F1203181F1E89446
:100870006F936E7F6E5F7F4F8F4F9F4FAF4FB1E093
:100880003ED0B4E03CD0670F781F891F9A1FA11D8E
:10089000680F791F8A1F911DA11D6A0F711D811D8F
:1008A000911DA11D20D009F468943F912AE0269F54
:1008B00011243019305D3193DEF6CF010895462FB3
:1008C0004770405D4193B3E00FD0C9F7F6CF462F94
:1008D0004F70405D4A3318F0495D31FD40524193FD
:1008E00002D0A9F7EACFB4E0A695979587957795BA
:1008F0006795BA95C9F700976105710508959B0141
:10090000AC010A2E06945795479537952795BA95C9
:10091000C9F7620F731F841F951FA01D0895F894D7
:02092000FFCF07
:0A092200FFFF25640079656574008D
:00000001FF
